******************************************************************************
               TMS320C6x Linker PC v6.1.12                     
******************************************************************************
>> Linked Thu Oct 28 14:13:30 2010

OUTPUT FILE NAME:   <timer_interrupt.out>
ENTRY POINT SYMBOL: "_c_int00"  address: 00808f60


MEMORY CONFIGURATION

         name            origin    length      used     unused   attr    fill
----------------------  --------  ---------  --------  --------  ----  --------
  L2                    00800000   000fffff  0000e0d6  000f1f29  RWIX
  MSM                   0c000000   001fffff  00000000  001fffff  RWIX


SECTION ALLOCATION MAP

 output                                  attributes/
section   page    origin      length       input sections
--------  ----  ----------  ----------   ----------------
.text      0    00800000    00009320     
                  00800000    00001800     Timer_Interrupt.obj (.text:csl_section:intc)
                  00801800    00000d20     Timer_Interrupt.obj (.text)
                  00802520    000007e0     rts64pluse.lib : divd.obj (.text:__divd)
                  00802d00    00000620     Timer_Interrupt.obj (.text:csl_section:tmr)
                  00803320    00000460     rts64pluse.lib : _printfi.obj (.text:__getarg_diouxp)
                  00803780    00000460                    : _printfi.obj (.text:__setfield)
                  00803be0    000003a0                    : _printfi.obj (.text:__printfi)
                  00803f80    00000320                    : _printfi.obj (.text:_fcvt)
                  008042a0    00000300                    : _printfi.obj (.text:_ecvt)
                  008045a0    00000300                    : fputs.obj (.text:_fputs)
                  008048a0    000002e0                    : _printfi.obj (.text:__pproc_fge)
                  00804b80    000002e0                    : _printfi.obj (.text:__pproc_fwp)
                  00804e60    00000280                    : _printfi.obj (.text:__pconv_e)
                  008050e0    00000280                    : memory.obj (.text:_free)
                  00805360    00000260                    : imath64.obj (.text:__divull)
                  008055c0    00000260                    : mpyd.obj (.text:__mpyd)
                  00805820    00000240                    : addd.obj (.text:__addd)
                  00805a60    00000220                    : _printfi.obj (.text:__pproc_diouxp)
                  00805c80    00000200                    : frcaddd.obj (.text:__frcaddd)
                  00805e80    00000200                    : frcmpyd_div.obj (.text:__frcmpyd_div)
                  00806080    00000200                    : _printfi.obj (.text:__pproc_str)
                  00806280    000001c0                    : _printfi.obj (.text:__mcpy)
                  00806440    000001a0                    : trgdrv.obj (.text:_HOSTrename)
                  008065e0    000001a0                    : imath40.obj (.text:__divul)
                  00806780    000001a0                    : setvbuf.obj (.text:_setvbuf)
                  00806920    00000180                    : _printfi.obj (.text:__pconv_g)
                  00806aa0    00000180                    : memory.obj (.text:_malloc)
                  00806c20    00000140                    : fputc.obj (.text:_fputc)
                  00806d60    00000140                    : lowlev.obj (.text:_getdevice)
                  00806ea0    00000140     _csl_intcIntrEnDisRes.obj (.text:csl_section:intc)
                  00806fe0    00000120     rts64pluse.lib : frcmpyd.obj (.text:__frcmpyd)
                  00807100    00000120                    : _printfi.obj (.text:__pproc_fflags)
                  00807220    00000120                    : fclose.obj (.text:_fclose)
                  00807340    00000100                    : trgdrv.obj (.text:_HOSTlseek)
                  00807440    00000100                    : _printfi.obj (.text:__ltostr)
                  00807540    00000100                    : _io_perm.obj (.text:__wrt_ok)
                  00807640    000000e0                    : trgdrv.obj (.text:_HOSTopen)
                  00807720    000000e0                    : autoinit.obj (.text:__auto_init)
                  00807800    000000e0                    : cmpd.obj (.text:__cmpd)
                  008078e0    000000e0                    : _printfi.obj (.text:__div)
                  008079c0    000000e0                    : atoi.obj (.text:_atoi)
                  00807aa0    000000e0                    : lowlev.obj (.text:_close)
                  00807b80    000000e0                    : exit.obj (.text:_exit)
                  00807c60    000000e0                    : memset.obj (.text:_memset)
                  00807d40    000000c0                    : trgdrv.obj (.text:_HOSTread)
                  00807e00    000000c0                    : trgdrv.obj (.text:_HOSTunlink)
                  00807ec0    000000c0                    : trgdrv.obj (.text:_HOSTwrite)
                  00807f80    000000c0                    : fopen.obj (.text:__cleanup)
                  00808040    000000c0                    : divu.obj (.text:__divu)
                  00808100    000000c0                    : fflush.obj (.text:__doflush)
                  008081c0    000000c0                    : fseek.obj (.text:_fseek)
                  00808280    000000c0                    : lowlev.obj (.text:_lseek)
                  00808340    000000c0                    : ltoa.obj (.text:_ltoa)
                  00808400    000000c0                    : lowlev.obj (.text:_write)
                  008084c0    000000a0                    : trgdrv.obj (.text:_HOSTclose)
                  00808560    000000a0                    : imath40.obj (.text:__divli)
                  00808600    000000a0                    : _printfi.obj (.text:__ecpy)
                  008086a0    000000a0                    : _printfi.obj (.text:__fcpy)
                  00808740    000000a0                    : fixdli.obj (.text:__fixdli)
                  008087e0    000000a0                    : _printfi.obj (.text:__pconv_f)
                  00808880    000000a0                    : lowlev.obj (.text:_finddevice)
                  00808920    000000a0                    : memcpy64.obj (.text:_memcpy)
                  008089c0    000000a0                    : memory.obj (.text:_minsert)
                  00808a60    000000a0                    : memory.obj (.text:_mremove)
                  00808b00    000000a0                    : printf.obj (.text:_printf)
                  00808ba0    00000080                    : fixdi.obj (.text:__fixdi)
                  00808c20    00000080                    : fltlid.obj (.text:__fltlid)
                  00808ca0    00000080                    : llshift.obj (.text:__llshl)
                  00808d20    00000080                    : renormd.obj (.text:__renormd)
                  00808da0    00000080                    : lowlev.obj (.text:_unlink)
                  00808e20    00000080                    : trgmsg.obj (.text:_writemsg)
                  00808ea0    00000060                    : llshift.obj (.text:__llshru)
                  00808f00    00000060                    : imath64.obj (.text:__subcull)
                  00808f60    00000060                    : boot.obj (.text:_c_int00)
                  00808fc0    00000060                    : memccpy.obj (.text:_memccpy)
                  00809020    00000060                    : trgmsg.obj (.text:_readmsg)
                  00809080    00000040                    : isinf.obj (.text:___isinf)
                  008090c0    00000040                    : _printfi.obj (.text:___isnan)
                  00809100    00000040                    : divd.obj (.text:___isnan)
                  00809140    00000040                    : args_main.obj (.text:__args_main)
                  00809180    00000040                    : negd.obj (.text:__negd)
                  008091c0    00000040                    : imath40.obj (.text:__remli)
                  00809200    00000040                    : subd.obj (.text:__subd)
                  00809240    00000020                    : negll.obj (.text:__negll)
                  00809260    00000020                    : _lock.obj (.text:__nop)
                  00809280    00000020                    : printf.obj (.text:__outc)
                  008092a0    00000020                    : printf.obj (.text:__outs)
                  008092c0    00000020                    : exit.obj (.text:_abort)
                  008092e0    00000020                    : remove.obj (.text:_remove)
                  00809300    00000020     _csl_intcNmiDummy.obj (.text:csl_section:intc)

.stack     0    00809320    00002000     UNINITIALIZED
                  00809320    00000008     rts64pluse.lib : boot.obj (.stack)
                  00809328    00001ff8     --HOLE--

.sysmem    0    0080b320    00002000     UNINITIALIZED
                  0080b320    00000008     rts64pluse.lib : memory.obj (.sysmem)
                  0080b328    00001ff8     --HOLE--

.far       0    0080d320    000004e8     UNINITIALIZED
                  0080d320    00000194     rts64pluse.lib : defs.obj (.far)
                  0080d4b4    00000004                    : fopen.obj (.far)
                  0080d4b8    00000190     Timer_Interrupt.obj (.far)
                  0080d648    000000d0     rts64pluse.lib : trgdrv.obj (.far)
                  0080d718    000000cc                    : lowlev.obj (.far)
                  0080d7e4    0000000c                    : exit.obj (.far)
                  0080d7f0    00000008                    : _lock.obj (.far)
                  0080d7f8    00000008                    : divd.obj (.far)
                  0080d800    00000008                    : memory.obj (.far)

.const     0    0080d808    0000033e     
                  0080d808    000001f8     Timer_Interrupt.obj (.const:.string)
                  0080da00    00000101     rts64pluse.lib : ctype.obj (.const:__ctypes_)
                  0080db01    00000023                    : _printfi.obj (.const:.string)
                  0080db24    00000002                    : fputs.obj (.const:.string)
                  0080db26    00000002     --HOLE-- [fill = 0]
                  0080db28    0000001e     csl_version.obj (.const:csl_section:version)

.switch    0    0080db48    00000084     
                  0080db48    00000084     Timer_Interrupt.obj (.switch)

.csl_vect 
*          0    0080dc00    00000200     
                  0080dc00    00000200     _csl_intcIsrDispatch.obj (.csl_vect)

.cinit     0    0080de00    00000194     
                  0080de00    0000005c     rts64pluse.lib : defs.obj (.cinit)
                  0080de5c    00000004     --HOLE-- [fill = 0]
                  0080de60    0000005c                    : lowlev.obj (.cinit)
                  0080debc    00000004     --HOLE-- [fill = 0]
                  0080dec0    0000002c     Timer_Interrupt.obj (.cinit)
                  0080deec    00000004     --HOLE-- [fill = 0]
                  0080def0    0000002c     rts64pluse.lib : exit.obj (.cinit)
                  0080df1c    00000004     --HOLE-- [fill = 0]
                  0080df20    0000002c                    : memory.obj (.cinit)
                  0080df4c    00000004     --HOLE-- [fill = 0]
                  0080df50    0000001c                    : _lock.obj (.cinit)
                  0080df6c    00000004     --HOLE-- [fill = 0]
                  0080df70    00000010                    : divd.obj (.cinit)
                  0080df80    0000000c                    : fopen.obj (.cinit)
                  0080df8c    00000004     --HOLE-- [fill = 0]
                  0080df90    00000004     (.pad.cinit) [fill = 0]

.cio       0    0080df98    00000120     UNINITIALIZED
                  0080df98    00000120     rts64pluse.lib : trgmsg.obj (.cio)

.bss       0    0080e0b8    00000058     UNINITIALIZED
                  0080e0b8    00000054     Timer_Interrupt.obj (.bss:csl_section:intc)
                  0080e10c    00000004     Timer_Interrupt.obj (.bss)


GLOBAL SYMBOLS: SORTED ALPHABETICALLY BY Name 

address    name
--------   ----
0080e0b8   $bss
0080e0b8   .bss
00800000   .text
008092c0   C$$EXIT
00808e80   C$$IO$$
00806f58   _CSL_intcGlobalDisable
00806f38   _CSL_intcGlobalEnable
00806fcc   _CSL_intcGlobalExcepClear
00806fa4   _CSL_intcGlobalExcepEnable
00806fb8   _CSL_intcGlobalExtExcepEnable
00806f90   _CSL_intcGlobalNmiEnable
00806f78   _CSL_intcGlobalRestore
00801118   _CSL_intcHookIsr
0080114c   _CSL_intcHwControl
008014b8   _CSL_intcInit
00806ef0   _CSL_intcInterruptClear
00806ed0   _CSL_intcInterruptDisable
00806eb0   _CSL_intcInterruptEnable
00806f0c   _CSL_intcInterruptRestore
00806f00   _CSL_intcInterruptSet
00801334   _CSL_intcOpen
008016e4   _CSL_intcPlugEventHandler
00806f24   _CSL_intcQueryInterruptStatus
00803224   _CSL_tmrGetBaseAddress
00802d14   _CSL_tmrHwControl
00802f0c   _CSL_tmrHwSetup
00802d00   _CSL_tmrInit
00802e50   _CSL_tmrOpen
0080db28   _CSL_versionStr
0080d558   _EventHandler
008084c0   _HOSTclose
00807340   _HOSTlseek
00807640   _HOSTopen
00807d40   _HOSTread
00806440   _HOSTrename
00807e00   _HOSTunlink
00807ec0   _HOSTwrite
0080df98   __CIOBUF_
0080e0b8   __CSL_intcAllocMask
0080e0c0   __CSL_intcCpuIntrTable
00800000   __CSL_intcDispatcher
008003b4   __CSL_intcEvent0Dispatcher
00800718   __CSL_intcEvent1Dispatcher
00800a70   __CSL_intcEvent2Dispatcher
00800dc8   __CSL_intcEvent3Dispatcher
0080e104   __CSL_intcEventHandlerRecord
0080e108   __CSL_intcEventOffsetMap
00806ea0   __CSL_intcIvpSet
00809300   __CSL_intcNmiDummy
0080e0bc   __CSL_intcNumEvents
0080dc00   __CSL_intcVectorTable
00002000   __STACK_SIZE
00002000   __SYSMEM_SIZE
0080d7ec   ___TI_enable_exit_profile_output
ffffffff   ___TI_pprof_out_hndl
ffffffff   ___TI_prof_data_size
ffffffff   ___TI_prof_data_start
ffffffff   ___binit__
0080e0b8   ___bss__
ffffffff   ___c_args__
0080de00   ___cinit__
0080e110   ___end__
00809320   ___etext__
00809080   ___isinf
ffffffff   ___pinit__
00800000   ___text__
00805820   __addd
00809140   __args_main
00807720   __auto_init
00807f80   __cleanup
0080d7e4   __cleanup_ptr
00807800   __cmpd
0080da00   __ctypes_
00802520   __divd
00808560   __divli
00808040   __divu
008065e0   __divul
00805360   __divull
00808100   __doflush
0080d7e8   __dtors_ptr
00808ba0   __fixdi
00808740   __fixdli
00808c20   __fltlid
00805c80   __frcaddd
00806fe0   __frcmpyd
00805e80   __frcmpyd_div
0080d4b0   __ft_end
0080d320   __ftable
00808ca0   __llshl
00808ea0   __llshru
0080d7f0   __lock
008055c0   __mpyd
00809180   __negd
00809240   __negll
00809260   __nop
00803be0   __printfi
008091c0   __remli
00808d20   __renormd
00809320   __stack
00808f00   __subcull
00809200   __subd
0080b320   __sys_memory
0080d410   __tmpnams
0080d7f4   __unlock
00807540   __wrt_ok
008092c0   _abort
008079c0   _atoi
00808f60   _c_int00
00807aa0   _close
0080d4c0   _context
00807b80   _exit
00807220   _fclose
00806c20   _fputc
008045a0   _fputs
008050e0   _free
008081c0   _fseek
00808280   _lseek
00808340   _ltoa
00802440   _main
00806aa0   _malloc
00808fc0   _memccpy
00808920   _memcpy
00807c60   _memset
00808b00   _printf
00806c20   _putc
00809020   _readmsg
008092e0   _remove
00806780   _setvbuf
0080e10c   _timerISRCounter
0080d4b8   _tmrIntcObj
00808da0   _unlink
00808400   _write
00808e20   _writemsg
ffffffff   binit
0080de00   cinit
0080e110   end
00809320   etext
ffffffff   pinit


GLOBAL SYMBOLS: SORTED BY Symbol Address 

address    name
--------   ----
00002000   __STACK_SIZE
00002000   __SYSMEM_SIZE
00800000   .text
00800000   __CSL_intcDispatcher
00800000   ___text__
008003b4   __CSL_intcEvent0Dispatcher
00800718   __CSL_intcEvent1Dispatcher
00800a70   __CSL_intcEvent2Dispatcher
00800dc8   __CSL_intcEvent3Dispatcher
00801118   _CSL_intcHookIsr
0080114c   _CSL_intcHwControl
00801334   _CSL_intcOpen
008014b8   _CSL_intcInit
008016e4   _CSL_intcPlugEventHandler
00802440   _main
00802520   __divd
00802d00   _CSL_tmrInit
00802d14   _CSL_tmrHwControl
00802e50   _CSL_tmrOpen
00802f0c   _CSL_tmrHwSetup
00803224   _CSL_tmrGetBaseAddress
00803be0   __printfi
008045a0   _fputs
008050e0   _free
00805360   __divull
008055c0   __mpyd
00805820   __addd
00805c80   __frcaddd
00805e80   __frcmpyd_div
00806440   _HOSTrename
008065e0   __divul
00806780   _setvbuf
00806aa0   _malloc
00806c20   _fputc
00806c20   _putc
00806ea0   __CSL_intcIvpSet
00806eb0   _CSL_intcInterruptEnable
00806ed0   _CSL_intcInterruptDisable
00806ef0   _CSL_intcInterruptClear
00806f00   _CSL_intcInterruptSet
00806f0c   _CSL_intcInterruptRestore
00806f24   _CSL_intcQueryInterruptStatus
00806f38   _CSL_intcGlobalEnable
00806f58   _CSL_intcGlobalDisable
00806f78   _CSL_intcGlobalRestore
00806f90   _CSL_intcGlobalNmiEnable
00806fa4   _CSL_intcGlobalExcepEnable
00806fb8   _CSL_intcGlobalExtExcepEnable
00806fcc   _CSL_intcGlobalExcepClear
00806fe0   __frcmpyd
00807220   _fclose
00807340   _HOSTlseek
00807540   __wrt_ok
00807640   _HOSTopen
00807720   __auto_init
00807800   __cmpd
008079c0   _atoi
00807aa0   _close
00807b80   _exit
00807c60   _memset
00807d40   _HOSTread
00807e00   _HOSTunlink
00807ec0   _HOSTwrite
00807f80   __cleanup
00808040   __divu
00808100   __doflush
008081c0   _fseek
00808280   _lseek
00808340   _ltoa
00808400   _write
008084c0   _HOSTclose
00808560   __divli
00808740   __fixdli
00808920   _memcpy
00808b00   _printf
00808ba0   __fixdi
00808c20   __fltlid
00808ca0   __llshl
00808d20   __renormd
00808da0   _unlink
00808e20   _writemsg
00808e80   C$$IO$$
00808ea0   __llshru
00808f00   __subcull
00808f60   _c_int00
00808fc0   _memccpy
00809020   _readmsg
00809080   ___isinf
00809140   __args_main
00809180   __negd
008091c0   __remli
00809200   __subd
00809240   __negll
00809260   __nop
008092c0   C$$EXIT
008092c0   _abort
008092e0   _remove
00809300   __CSL_intcNmiDummy
00809320   ___etext__
00809320   __stack
00809320   etext
0080b320   __sys_memory
0080d320   __ftable
0080d410   __tmpnams
0080d4b0   __ft_end
0080d4b8   _tmrIntcObj
0080d4c0   _context
0080d558   _EventHandler
0080d7e4   __cleanup_ptr
0080d7e8   __dtors_ptr
0080d7ec   ___TI_enable_exit_profile_output
0080d7f0   __lock
0080d7f4   __unlock
0080da00   __ctypes_
0080db28   _CSL_versionStr
0080dc00   __CSL_intcVectorTable
0080de00   ___cinit__
0080de00   cinit
0080df98   __CIOBUF_
0080e0b8   $bss
0080e0b8   .bss
0080e0b8   __CSL_intcAllocMask
0080e0b8   ___bss__
0080e0bc   __CSL_intcNumEvents
0080e0c0   __CSL_intcCpuIntrTable
0080e104   __CSL_intcEventHandlerRecord
0080e108   __CSL_intcEventOffsetMap
0080e10c   _timerISRCounter
0080e110   ___end__
0080e110   end
ffffffff   ___TI_pprof_out_hndl
ffffffff   ___TI_prof_data_size
ffffffff   ___TI_prof_data_start
ffffffff   ___binit__
ffffffff   ___c_args__
ffffffff   ___pinit__
ffffffff   binit
ffffffff   pinit

[138 symbols]
